:100000000C9434000C9462040C9446000C9446004A
:100010000C9446000C9446000C9446000C94460048
:100020000C9446000C9446000C9446000C94460038
:100030000C9446000C9446000C9446000C94460028
:100040000C9446000C9446000C9446000C94460018
:100050000C9446000C9446000C9446000C94460008
:100060000C9446000C94460011241FBECFEFD8E03C
:10007000DEBFCDBF11E0A0E0B1E001C01D92A4320F
:10008000B107E1F70E94FB020C946C040C94000091
:1000900040EA5FE009C020E0FA013197F1F72F5FF5
:1000A0002F3FD1F78F5F90408F3F910509F098F770
:1000B000009749F020E040EA5FE0FA013197F1F75C
:1000C0002F5F2817D0F30895569A5E9884B58C7BDD
:1000D00084BD84B5816884BD089581E0603078076F
:1000E00001F181E06130780750F468307105A9F0C2
:1000F00060347105A1F061307105D9F40CC08FEF47
:100100006E3F7807A1F08FEF6F3F780770F4605073
:10011000744079F408C081E10DC082E10BC083E135
:1001200009C084E107C085E105C086E103C087E11D
:1001300001C080E185BD0895229883B1847090E06C
:100140009595879595958795982F811191E0492FE1
:1001500020E030E060EA7FE006C02F5F3F4F2A30AA
:100160003105A0F4492FCB010197F1F7229883B113
:10017000847090E09595879595958795982F811136
:1001800091E0941751F320E030E0ECCF892F0895EF
:10019000579889B1807890E0880F892F881F990B34
:1001A000982F811191E0492F20E030E060EA7FE054
:1001B00006C02F5F3F4F2A303105A0F4492FCB01F5
:1001C0000197F1F7579889B1807890E0880F892FCF
:1001D000881F990B982F811191E0941751F320E01B
:1001E00030E0ECCF892F0895529889B1847090E067
:1001F0009595879595958795982F811191E0492F31
:1002000020E030E060EA7FE006C02F5F3F4F2B30F8
:100210003105A0F4492FCB010197F1F7529889B12C
:10022000847090E09595879595958795982F811185
:1002300091E0941751F320E030E0ECCF892F08953E
:1002400081E0809309018FEF90E061E070E00E940F
:100250006D000E94640008950E94C800811181E031
:100260008093000180EA9FE0FC013197F1F701974C
:10027000F1F780910001882321F481E0809303014C
:100280000895109203010895549A5C9A10920B01FC
:1002900090910B0180910901811197BD569A80912F
:1002A0000B01882311F05E9A01C05E988BB120E0AB
:1002B00040EA5FE0CA010197F1F72F5F2A3FD1F7CB
:1002C00020E040EA5FE0CA010197F1F72F5F2A3F83
:1002D000D1F720E040EA5FE0CA010197F1F72F5F14
:1002E0002A3FD1F720E040EA5FE0CA010197F1F729
:1002F0002F5F2A3FD1F7549A5C980895559A5D9ADA
:1003000084EF91E00E944800559A5D9884EF91E057
:100310000E944800559A5D9A84EF91E00E9448003F
:10032000559A5D9884EF91E00E944800559A5D9A35
:1003300084EF91E00E944800559A5D9884EF91E027
:100340000E94480008958AE080930B0190910B0170
:1003500080910901811197BD8CE291E00E944800D3
:1003600084E180930B0190910B018091090181112F
:1003700097BD8CE291E00E9448008EE180930B01D2
:1003800090910B0180910901811197BD8CE291E060
:100390000E94480082E380930B0190910B018091B1
:1003A0000901811197BD8CE291E00E94480086E42A
:1003B00080930B0190910B0180910901811197BDF0
:1003C0008CE291E00E94480084E680930B019091BA
:1003D0000B0180910901811197BD8CE291E00E948F
:1003E00048008EE680930B0190910B0180910901EA
:1003F000811197BD8CE291E00E94480082E88093D1
:100400000B0190910B0180910901811197BD8CE244
:1004100091E00E94480086E980930B0190910B01C6
:1004200080910901811197BD8CE291E00E94480002
:1004300084EB80930B0190910B0180910901811154
:1004400097BD8CE291E00E9448008CED80930B01F7
:1004500090910B0180910901811197BD8CE291E08F
:100460000E9448008EEF80930B0190910B018091C8
:100470000901811197BD8CE291E00E944800089526
:1004800081E08093060110920401209A8091060178
:10049000882311F0289A01C0289885B1219A80916B
:1004A0000401882311F0299A01C0299885B1569A30
:1004B00080910B01882311F05E9A01C05E988BB188
:1004C00008951092060181E080930401209A8091A2
:1004D0000601882311F0289A01C0289885B1219A35
:1004E00080910401882311F0299A01C0299885B1CF
:1004F000569A80910B01882311F05E9A01C05E9894
:100500008BB10895259A2D9A84EF91E00E944800BE
:10051000259A2D9884EF91E00E9448000895549AFE
:100520005C9A84EF91E00E944800549A5C9884EFB2
:1005300091E00E944800549A5C9A84EF91E00E94F6
:100540004800549A5C9884EF91E00E944800549AC5
:100550005C9A84EF91E00E944800549A5C9884EF82
:1005600091E00E94480008950E949C00811181E062
:100570008093070180EA9FE0FC013197F1F7019732
:10058000F1F780910701882321F482E08093030131
:1005900008951092030108958FEF84B915B88AB9B0
:1005A0001BB887B918B8229883B1847090E09595EC
:1005B000879595958795982F811191E090930001EB
:1005C000579889B1807890E0880F892F881F990B00
:1005D000982F811191E090930701529889B184700E
:1005E00090E09595879595958795982F811191E045
:1005F0009093050108951F93CF93DF9314BE14BE0B
:1006000088E10FB6F89480936000109260000FBEEE
:100610000E94CC020E9482020E947E010E94200160
:100620000E948F02109202011092010110920B01A0
:10063000109205011092030110920601109204011C
:10064000109202011092010110920B018091690039
:100650008360809369007894E89AC0EADFE011E053
:100660000E94F400811181E08093050120E0CE0119
:100670000197F1F72F5F2A30D1F780910501882388
:1006800009F4FDC00E942C0180910301813009F022
:10069000EFC00E946102559A5D9A0E94A3011092D8
:1006A000080143C0549A5C9820E0CE010197F1F70D
:1006B0002F5F2436D1F70E94B4028091030182306B
:1006C00059F50E944401559A5D98549A5C9A30E01D
:1006D0001EC0CE010197F1F72F5F2A3FD1F720E02E
:1006E000CE010197F1F72F5F2A3FD1F720E0CE012D
:1006F0000197F1F72F5F2A3FD1F720E0CE01019754
:10070000F1F72F5F2A3FD1F73F5F323011F020E041
:10071000E0CF1093080109C0549A5C9A20E0CE0102
:100720000197F1F72F5F2436D1F7809108018823D4
:1007300009F4B8CF1092080110920301549A5C9802
:1007400030E041C0549A5C9A559A5D9A20E0CE01FF
:100750000197F1F72F5F2A3FD1F720E0CE010197F3
:10076000F1F72F5F2A3FD1F720E0CE010197F1F793
:100770002F5F2A3FD1F720E0CE010197F1F72F5FDD
:100780002A3FD1F7549A5C98559A5D9820E0CE01A3
:100790000197F1F72F5F2A3FD1F720E0CE010197B3
:1007A000F1F72F5F2A3FD1F720E0CE010197F1F753
:1007B0002F5F2A3FD1F720E0CE010197F1F72F5F9D
:1007C0002A3FD1F73F5F3E3108F4BCCF30930A0196
:1007D000549A5C98559A5D9A0E9440020E94A30127
:1007E00041C0549A5C9820E0CE010197F1F72F5F49
:1007F0002436D1F70E942C0180910301813049F504
:100800000E944401549A5C9A30E01EC0CE010197C8
:10081000F1F72F5F2A3FD1F720E0CE010197F1F7E2
:100820002F5F2A3FD1F720E0CE010197F1F72F5F2C
:100830002A3FD1F720E0CE010197F1F72F5F2A3F41
:10084000D1F73F5F323011F020E0E0CF1093080184
:1008500009C0549A5C9A20E0CE010197F1F72F5F0E
:100860002436D1F780910801882309F4BACF02C059
:100870000E948F02559A5D98259A2D9806C0549A29
:100880005C9A80E991E00E944800549A5C9810922A
:1008900005011092030110920601109204011092BA
:1008A00002011092010110920B0183B7817F8660D3
:1008B00083BF83B7816083BF7894889583B78E7F29
:1008C00083BFCECE1F920F920FB60F9211240F90BE
:0C08D0000FBE0F901F901895F894FFCFFA
:00000001FF
